:020000040800F2
:1000000090340020050100085115000887070008FA
:100010004D1500084D070008351B000800000000C2
:10002000000000000000000000000000A11800080F
:100030008507000800000000A1170008A3180008A9
:100040001F0100081F0100081F0100081F01000810
:100050001F0100081F0100081F0100081F01000800
:100060001F0100081F0100081F0100081F010008F0
:100070001F0100081F010008650700087507000838
:100080001F0100081F0100081F0100081F010008D0
:100090001F0100081F0100081F0100081F010008C0
:1000A0001F010008991900081F0100081F0100081E
:1000B0001F010008691A00081F0100081F0100083D
:1000C0001F0100081F0100081F0100081F01000890
:1000D0001F010008251B00081F0100081F01000860
:1000E0001F0100081F0100081F010008DFF810D0E1
:1000F00000F01AFB00480047B12B0008AFF3008066
:10010000903400200648804706480047FEE7FEE797
:10011000FEE7FEE7FEE7FEE7FEE7FEE7FEE7FEE7B7
:1001200095190008ED000008D2B201E000F8012B9B
:10013000491EFBD270470022F6E710B513460A4667
:1001400004461946FFF7F0FF204610BD421C10F888
:10015000011B0029FBD1801A7047F0B480EA01022C
:10016000D40F4200B2EB410F02D2024608461146BC
:100170004A0042D0C30DDDB2C1F3C752AD1A202DE3
:1001800035DAC1F3160141F4000204B15242C5F15F
:10019000200602FA06F12A411044B3EBD05F23D0C7
:1001A000C4B1012DA0EBC35009DCF0BC4FF00042FC
:1001B00002EAC352DBB200F5000000F02ABA4000A8
:1001C00000F1807000EBC350A0F1807040EAD17064
:1001D000490009E0490841EAC071A0EBC35000F5AD
:1001E0000000400800EBC350F0BC00F009BA6142C7
:1001F000012202EB4101001BF6E7F0BC704781F0E1
:100200000041AAE780F00040A7E780EA010210B5AC
:1002100002F00043400022D04A001FD0010E01EB43
:100220001261C0F35600C2F3560240F4000042F4DB
:100230000002A0FB022000047F39140400D0401CFF
:1002400050EA124001D44000491EC2B20C0604EB31
:10025000D010401C4008802A02D003E0002010BDCE
:1002600020F00100002900DA0020184310BD30B44E
:1002700080EA010202F0004530F0004221F0004027
:1002800013D090B1C30DD40DC2F31601C0F3160004
:10029000E41A41F4000140F400027D34914201D39C
:1002A000641C00E04900002C02DA30BC00207047DA
:1002B0004FF400000023914201D3891A0343400800
:1002C0004FEA4101F7D151B1914202D14FF00041C3
:1002D00005E002D24FF0010101E06FF0010103EBF4
:1002E000C450284430BC00F08BB92DE9FE4F804645
:1002F00081EA0300C00F0C46009021F0004123F07A
:100300000045B8EB0200A94105D24046214690467F
:100310001C460B46024623F00040104347D0270DF1
:10032000C7F30A00C3F30A510290401A0190402813
:100330006BDAC3F3130040F4801B0098924620B19F
:100340000023D2EB030A63EB0B0B01985946C0F173
:100350004002504600F023F906460D4650465946E5
:10036000019A00F03BF910EB08006141002487EA94
:10037000115284EAE7731A4340D0009A62B3019A9B
:10038000012A4FEA075215DC001B61EB02014FF016
:10039000004202EA0752CDE90042001C41F58011FB
:1003A00032462B4600F072F903B0BDE8F08F4046AC
:1003B0002146F9E7001B61EB0201001C41F58013A7
:1003C00000185B412018A2F5001747EB030140EA33
:1003D000D570B6196D4111E06D084FEA360645EA51
:1003E000C0754FEA0752001B61EB0201001C41F58A
:1003F000801149084FEA30000019514132462B461E
:1004000003B0BDE8F04F00F032B90098012240007F
:100410000023D0EB020263EBE073009821464FEA21
:10042000E074B8EB000061EB0401E9E783F00043FE
:100430005BE781F0004158E7C10F80EAE0700844B3
:10044000CA079623002100F0E4B896230022114643
:1004500000F0DFB800F0004220F00040C10DC0F312
:10046000160040F400007F2901DA00207047962929
:1004700003DCC1F19601C84001E096398840002AAA
:10048000F4D04042704720F00040C10DC0F3160088
:1004900040F400007F2901DA00207047962903DC30
:1004A000C1F19601C840704796398840704770B5D1
:1004B000C1F30A5201F000450024C1F3130140F2D8
:1004C000FF3341F480119A4201DA002070BD40F2FE
:1004D00033439A42A2F2334203DC524200F06EF8F8
:1004E00000E090402C43F1D0404270BD00F000424B
:1004F00030F000400AD0C10D01F56071C0F3160064
:1005000042EA0151C20840071143704700200146EA
:1005100070470000002801DBC0F10040002901DB2A
:10052000C1F1004181427047002801DBC0F1004069
:10053000002901DBC1F10041884270472DE9F05FDD
:100540000546002092469B46884606468146402442
:100550001BE0284641464746224600F02FF8534606
:100560005A46C01A914110D311461846224600F04F
:1005700016F82D1A67EB01084F462246012000218C
:1005800000F00DF817EB00094E41201EA4F1010404
:10059000DFDC484631462A464346BDE8F09F202A24
:1005A00004DB203A00FA02F1002070479140C2F1CA
:1005B000200320FA03F3194390407047202A04DBFC
:1005C000203A21FA02F00021704721FA02F3D040CC
:1005D000C2F120029140084319467047202A06DBE9
:1005E000CB17203A41FA02F043EAE07306E041FA01
:1005F00002F3D040C2F120029140084319467047EF
:100600000029A8BF7047401C490008BF20F0010026
:10061000704710B4B0FA80FC00FA0CF050EA010404
:1006200004BF10BC704749B1CCF1200421FA04F496
:1006300011FA0CF118BF012121430843A3EB0C016F
:10064000CB1D4FEA00614FEA102042BF002010BCD2
:10065000704700EBC35010440029A4BF10BC704782
:10066000401C490008BF20F0010010BC704710B5C5
:10067000141E73F1000408DA401C41F100019218C5
:100680005B411A4301D120F0010010BD2DE9F04D6E
:1006900092469B4611B1B1FA81F202E0B0FA80F2C3
:1006A00020329046FFF77BFF04460F4640EA0A00DF
:1006B00041EA0B0153465A46084313D0114653EA08
:1006C000010019D0C8F140025046FFF777FF0546F8
:1006D0000E46504659464246FFF761FF084305D093
:1006E000012004E020463946BDE8F08D0020054396
:1006F00046EAE0762C4337430A986305E40AA0EB08
:1007000008000022FD0A44EA47540A3002D50020BE
:100710000146E9E7010510196941DDE908450019BD
:100720006941BDE8F04DA2E7064C074D06E0E068E0
:1007300040F0010394E8070098471034AC42F6D328
:10074000FFF7D8FC94540008B454000800BFFEE73B
:10075000024600BF1AB901E000BF00BFFCE700BFBE
:100760000120704710B50248006803F034FD10BD49
:100770005C00002010B50248006803F02CFD10BD9D
:100780005C000020704700BFFEE7000008B5054987
:10079000C9690143034AD1611146C9690140009109
:1007A00000BF08BD0010024008B505498969014332
:1007B000034A9161114689690140009100BF08BD5B
:1007C0000010024008B5054989690143034A916157
:1007D000114689690140009100BF08BD0010024028
:1007E00008B5054989690143034A91611146896940
:1007F0000140009100BF08BD0010024008B5054946
:1008000089690143034A9161114689690140009158
:1008100000BF08BD0010024010B54A1E044B9A5C90
:10082000825822F001034A1E014CA25C835010BD85
:10083000CC47000810B54A1E044B9A5C825842F01F
:1008400001034A1E014CA25C835010BDCC47000836
:1008500010B54A1E044B9A5C825842F002034A1EAD
:10086000014CA25C835010BDCC47000830B54B1E34
:10087000054CE35CC35823F4405313434C1E024D14
:100880002C5D035130BD00008A47000830B54B1E77
:10089000064CE35C03445B686FF30F0313434C1E89
:1008A000024D2C5D0444636030BD0000CC4700085D
:1008B00030B54B1E054CE35CC35844F21004A3430F
:1008C00013434C1E014D2C5D035130BD8A47000877
:1008D00010B54B1E024CE35C0344DA6010BD00000F
:1008E000CC47000830B54B1E054CE35CC35823F0E1
:1008F000800313434C1E024D2C5D035130BD00009C
:100900008A47000830B54B1E054CE35CC35823F4FE
:10091000406313434C1E024D2C5D035130BD00005B
:100920008A47000830B54B1E054CE35CC35823F0E2
:10093000200313434C1E024D2C5D035130BD0000BB
:100940008A47000810B54B1E024CE35C03449A60D2
:1009500010BD0000CC47000830B54B1E054CE35CD1
:10096000C35823F0400313434C1E024D2C5D03512A
:1009700030BD00008A47000830B54B1E054CE35CD3
:10098000C35823F4407313434C1E024D2C5D035196
:1009900030BD00008A4700082DE9F04102460B46B1
:1009A0001868C0F30F2595FAA5F0B0FA80F480E03E
:1009B0000120A040284000287AD0082C04D240F220
:1009C000011000FA04F106E0A4F108004FF001164E
:1009D000864046F08061586808280ED11869D668AC
:1009E00026EA11260F0A97FAA7F7B7FA87F700FA4F
:1009F00007F73E43D66000BF00BF586802EB1166A0
:100A000091FAA1FCBCFA8CFC4FEA8C084FF00F0C59
:100A10000CFA08FC376827EA0C0791FAA1FCBCFA2B
:100A20008CFC4FEA8C0C00FA0CFC47EA0C07376090
:100A300000BF5868012802D05868092838D1986842
:100A400002EB116691FAA1FCBCFA8CFC4FEA8C080F
:100A50004FF0030C0CFA08FC376827EA0C0791FAF0
:100A6000A1FCBCFA8CFC4FEA8C0C00FA0CFC47EAA7
:100A70000C07376000BFD86802EB116691FAA1FC41
:100A8000BCFA8CFC4FEA8C084FF0040C0CFA08FC02
:100A9000376827EA0C0791FAA1FCBCFA8CFC4FEAF4
:100AA0008C0C00FA0CFC47EA0C07376000BF00BF53
:100AB000641C25FA04F000287FF47AAFBDE8F081C9
:100AC00002469068C1F30F231840C1F30F239842E8
:100AD00001D1012070470020FCE7C1F30F224261E1
:100AE0007047C1F30F2242617047C1F30F22426188
:100AF0007047C1F30F220261704770B500EB1163BC
:100B000091FAA1F5B5FA85F5AE000F25B5401C6840
:100B1000AC4391FAA1F5B5FA85F5AD0002FA05F5F9
:100B20002C431C6070BD000002480068401C014955
:100B300008607047200000204FF47A71B0FBF1F29A
:100B4000521E4FF0E0235A6100229A6105221A6179
:100B500000BF704710B5044600F058FE20602068C2
:100B600000F020FE6060606800F02CFEA06060680D
:100B700000F03AFEE06010BD016841F04001016004
:100B8000704730B50246012300BF1068C0F38010E3
:100B900038BBD1E9000420438C682043CC68204353
:100BA0000C6920434C6920438C692043CC69204365
:100BB0000C6A204314684FF6BF75AC4320431060A5
:100BC000506820F004004C6940EA14405060086A04
:100BD000B0F5005F04D1486A84B2146100BF00BF61
:100BE0000023184630BD000001490860704700002E
:100BF00000000020016821F08001016070478168D9
:100C000021F0800181607047016841F001010160BD
:100C10007047C16841F00101C160704710B50246DC
:100C200013681C48824208D0B2F1804F05D01A48A0
:100C3000824202D01948824204D123F070004C68ED
:100C400040EA04031348824208D0B2F1804F05D035
:100C50001148824202D01148824204D123F44070EC
:100C6000CC6840EA040313608868D06200BF08883B
:100C7000906200BF0748824203D10869106300BF39
:100C800000BF00BF506940F00100506100BF00206C
:100C900010BD0000002C014000040040000800408E
:100CA00001460869C0F34000704701460869C0F377
:100CB0008000704701460869C0F3C00070470146D4
:100CC0000869C0F3001070470146086900F0010090
:100CD00070470146C868C0F3400070470146C868C5
:100CE000C0F3800070470146C868C0F3C000704779
:100CF0000146C868C0F3001070470146C86800F09C
:100D00000100704770B50246012901D1002416E0A8
:100D1000042901D1012412E0102901D102240EE09E
:100D2000402901D103240AE0B1F5807F01D10424D8
:100D300005E0B1F5806F01D1052400E006242346CB
:100D4000064CE55C02F1180428190468044DEE5CB9
:100D50000425B5402C43046070BD000067470008BF
:100D60006E47000870B50246012901D1002416E043
:100D7000042901D1012412E0102901D102240EE03E
:100D8000402901D103240AE0B1F5807F01D1042478
:100D900005E0B1F5806F01D1052400E0062423466B
:100DA000064CE55C02F1180428190468044DEE5C59
:100DB0000825B5402C43046070BD0000674700085B
:100DC0006E4700082DE9F04106460C4615460127FE
:100DD000012C08D0102C0CD0B4F5807F0FD0B4F5C6
:100DE000805F18D111E02946304600F0F3FB07463A
:100DF00012E02946304600F029FC07460CE029465F
:100E0000304600F065FC074606E02946304600F013
:100E10009BFC074600E000BF00BF3846BDE8F081FC
:100E200081637047826844F207039A430A438260F1
:100E30007047426822F070020A434260704708B56A
:100E40000168009100BF4168009100BF08BD6FF0CC
:100E500040010160704700002DE9FF4104460D4646
:100E600001270026204600F055F8002833D1E96814
:100E70006868084329690843E16841F20C629143BC
:100E80000843E060A868216921F4405101432161D1
:100E900000BF6869616921F440710143616100BF6D
:100EA0006846FFF757FE0E48844201D1039E08E0D2
:100EB0000C48844201D1029E03E00B48844200D1D9
:100EC000029E46B1286830B10027314620462A6884
:100ED00000F025F800BF384604B0BDE8F0810000FE
:100EE00000380140004400400048004001460868C6
:100EF000C0F34000704701460868C0F380007047A7
:100F000001460868C0F3C000704701460868C0F396
:100F1000801070470146C868C0F34030704770B514
:100F200001EBC10303EB01139400B3FBF4F301EBFA
:100F3000C10404EB01149500B4FBF5F46425B4FB83
:100F4000F5F404EBC40505EB0414A3EB840332248D
:100F500004EB03136424B3FBF4F303F0F00301EB9D
:100F6000C10404EB01149500B4FBF5F46425B4FB53
:100F7000F5F403EB041401EBC10303EB011395003B
:100F8000B3FBF5F301EBC10505EB01159600B5FBCD
:100F9000F6F56426B5FBF6F505EBC50606EB05157B
:100FA000A3EB8503322505EB03136425B3FBF5F3AF
:100FB00003F00F0323449BB2836070BD38B501205A
:100FC000144949690143134A516111464969014075
:100FD000009100BF00BF00F0E3FD0546002211466E
:100FE00000F0B8FA044621460E2000F0E9FD0E207C
:100FF00000F0BCFD00F0D4FD05460022114600F0D3
:10100000A9FA044621460F2000F0DAFD0F2000F077
:10101000ADFD38BD0010024000B585B01421684612
:10102000FFF789F81020FFF7BFFB2020FFF7BCFB7C
:101030000420FFF7B9FB0820FFF7B6FB3549364817
:10104000FFF74BFD41F618013448FFF746FD3449E0
:101050003448FFF742FD2F48009001200190022004
:1010600002900020039069462B48FFF795FC2E481C
:1010700000900020019069462748FFF78DFC2B481F
:1010800000900020019069462448FFF785FC40F657
:10109000080000900120019002200290002003909F
:1010A000049069461D48FFF777FC41F2100000905C
:1010B0000120019002200290002003900120049062
:1010C00069461648FFF768FC40F2033000900120A3
:1010D0000190022002900020039069461148FFF71A
:1010E0005BFC134800900020019069460D48FFF713
:1010F00053FC104800900120019003200290002032
:1011000003900120049069460648FFF745FC05B0AE
:1011100000BD000020002004001001400008014034
:1011200033033004000C0140C000C0049D05990445
:10113000FFFCCF043000300400B58FB0282105A893
:10114000FEF7F9FF14216846FEF7F5FF4FF48050D3
:10115000FFF738FB0420FFF735FB4AF2A0000090B0
:101160000920019003200290002003906946134853
:10117000FFF712FC44F24000009004200190694601
:101180000E48FFF709FC002005904FF4827006908E
:1011900000200790022008900120099040020A9048
:1011A00038200B9000200C900D900A200E9005A97D
:1011B0000348FFF7E6FC0FB000BD00000008014047
:1011C0000030014030B585B014216846FEF7B3FF0A
:1011D0004FF40060FFF704FB00F0EAFC0546002234
:1011E000032100F0D7F904462146192000F0FCFC49
:1011F000192000F0C8FC41F61F40ADF800000020A7
:1012000001906320029000200390049069460948F1
:10121000FFF704FD0748FFF7EDFC00210548FFF745
:1012200001FE00210348FFF704FE0248FFF7E7FC38
:1012300005B030BD002C014000B593B014210EA8BC
:10124000FEF779FF202106A8FEF775FF142101A8FB
:10125000FEF771FF0120FFF799FA0020ADF8380082
:101260000F9041F61F401090002011900EA94FF0F2
:101270008040FFF7D3FC00BF4FF08040006840F093
:1012800080004FF08041086000BF00214FF0804097
:10129000FFF7C8FD10218806FFF764FD7020069057
:1012A000002007900890099002200A9006AA1021B9
:1012B0004007FFF787FD10218806FFF723FD002177
:1012C0004FF08040FFF7B5FD4FF08040FFF797FCEF
:1012D0000420FFF785FA40F20220019009200290D5
:1012E000022003900020049001A90248FFF754FB5C
:1012F00013B000BD0008014030B585B01421684628
:10130000FEF719FF0220FFF741FA00F051FC0546F5
:101310000022032100F03EF9044621461D2000F082
:1013200063FC1D2000F02FFC41F61F40ADF80000CB
:101330000020019063200290002003906946094834
:10134000FFF76CFC0748FFF755FC00210548FFF745
:1013500069FD00210348FFF76CFD0248FFF74FFCD1
:1013600005B030BD000400402DE9F0418CB01C21D7
:1013700005A8FEF7E0FE14216846FEF7DCFE4FF4F8
:101380008040FFF73BFA0420FFF738FA68480090E6
:1013900009200190032002900020039069466548CF
:1013A000FFF7FAFA6448009004200190694661480A
:1013B000FFF7F2FA002205216048FFF779FA0022D0
:1013C00005215E48FFF752FA002205215B48FFF72E
:1013D000A9FA002205215948FFF7BEFA802205210B
:1013E0005648FFF77FFA002205215448FFF7C4FA58
:1013F000002205215148FFF785FA102204214F48A9
:10140000FFF756FA002204214C48FFF72FFA00227A
:1014100004214A48FFF786FA002204214748FFF7D3
:101420009BFA802204214548FFF75CFA0022042140
:101430004248FFF7A1FA002204214048FFF762FA70
:1014400025213F4B1B68C3F30220052400250346DA
:10145000C3F1070CBCF1040F02D94FF0040C01E0FA
:10146000C3F1070C674603F1040CBCF1070F02D26D
:101470004FF0000C01E0A3F1030C66464FF0010CA5
:101480000CFA07FCACF1010C0CEA040C0CFA06FC9B
:101490004FF0010808FA06F8A8F1010808EA050863
:1014A0004CEA080200BF002904DB1007030E2548A0
:1014B000435407E01007040E21480C3001F00F03DD
:1014C0001B1FC45400BF2520002809DB00F01F02A9
:1014D000012191404209920002F1E022C2F800117C
:1014E00000BF4FF4E130059000200690079008906F
:1014F0000C20099000200A900B9005A91248FFF7D4
:10150000ABFC00BF1048006920F490400E49086110
:101510000846406920F02A00486100BF00BF084625
:10152000C06840F40050C86000BF0CB0BDE8F08156
:10153000020002040008014004000404000002400C
:101540000CED00E000E400E00038014000BFFEE7E1
:1015500000BFFEE7F0B503460C4603F00701C1F1FA
:101560000700042801D9042001E0C1F10700064664
:10157000081D072801D2002000E0C81E05460120F2
:10158000B040401E2040A8400127AF407F1E1740BA
:101590003843F0BDF0B503460C4603F00701C1F136
:1015A0000700042801D9042001E0C1F10700064624
:1015B000081D072801D2002000E0C81E05460120B2
:1015C000B040401E2040A8400127AF407F1E17407A
:1015D0003843F0BD70B50246106A20F00100106279
:1015E000136A5568946924F0030424F070000E68AF
:1015F00040EA060423F002000E6940EA060323F0E5
:1016000001004E6840EA06030F48824213D123F0DE
:1016100008004E6940EA860323F004008E6840EA21
:10162000860325F480708E6940EA060525F4007073
:10163000CE6940EA460555609461C868506300BFB2
:101640001362002070BD0000002C01402DE9F04124
:1016500004460D46206A20F010002062266AD4F865
:101660000480A76927F4407727F4E040296840EA1E
:10167000012726F02000296940EA011626F0100013
:10168000696840EA01161148844213D126F08000AF
:10169000696940EA811626F04000A96840EA81168F
:1016A00028F48060A96940EA810828F40060E969AB
:1016B00040EAC108C4F80480A7612046E968FFF742
:1016C000AFFB26620020BDE8F0810000002C014045
:1016D00070B50246106A20F480701062136A556873
:1016E000D46924F0030424F070000E6840EA060474
:1016F00023F400700E6940EA062323F480704E68DC
:1017000040EA06230F48824213D123F400604E6959
:1017100040EA862323F480608E6840EA862325F41D
:1017200080508E6940EA061525F40050CE6940EAE3
:1017300046155560D461C868D06300BF13620020AD
:1017400070BD0000002C014070B50246106A20F404
:1017500080501062146A5568D36923F4407323F4EF
:10176000E0400E6840EA062324F400500E6940EA87
:10177000063424F480504E6840EA0634074882421A
:1017800004D125F480408E6940EA86155560D36106
:10179000C868106400BF1462002070BD002C0140B6
:1017A00070470000014600BF0448406800F0F000A8
:1017B0000009034A125C21FA02F07047001002404F
:1017C000B4470008014600BF0548406800F4E060E7
:1017D000044A02EB1020027821FA02F07047000060
:1017E00000100240C4470008014600BF0548406899
:1017F00000F46050044A02EBD020027821FA02F093
:101800007047000000100240C447000810B50024D3
:1018100000BF0B48406800F00C0020B1042804D041
:10182000082808D103E0074C07E0064C05E000F06B
:101830000BF8044601E0034C00BF00BF204610BD7A
:101840000010024000127A000021002200BF11485F
:10185000406800F4803002461AB1B2F5803F0CD1E6
:1018600001E00D490BE000BF0A484068C0F340406A
:10187000401C0A4BB3FBF0F101E0074900BF00BF79
:1018800000BF0448406800F47010022303EB90404E
:10189000484370470010024000093D0000127A00E2
:1018A0007047704710B502203749096821F00701D9
:1018B0000143354A116000BF00BF00BF32480068D5
:1018C00000F007000228F8D100BF3048006840F45B
:1018D00080302E49086000BF00BF00BF2B48006861
:1018E000C0F340400028F8D04FF480304FF4E011AE
:1018F000264A526822F47C1200F440330B431A4308
:10190000224B5A6000BF00BF1846006840F080704C
:101910001946086000BF00BF00BF1C480068C0F344
:1019200040600028F8D000201849496821F0F001F3
:101930000143164A516000BF10151146496821F451
:10194000E0610143516000BF00201146496821F465
:1019500060510143516000BF02201146496821F0E7
:1019600003010143516000BF00BF00BF074840684A
:1019700000F00C000828F8D10548FFF7DDF804480E
:10198000FFF732F910BD00000020024000100240B5
:1019900000A24A047047000010B53148FFF794F9DF
:1019A00001285CD100BF2E48FFF77AF901280AD13F
:1019B0002B48FFF78EF9012805D100BF001F2849E9
:1019C000086100BF00BF2648FFF76FF901280AD160
:1019D0002348FFF783F9012805D100BF801F204964
:1019E000086100BF00BF1E48FFF764F901280BD152
:1019F0001B48FFF778F9012806D100BF6FF00800F7
:101A00001749086100BF00BF1548FFF758F90128C2
:101A10000BD11348FFF76CF9012806D100BF6FF016
:101A200010000F49086100BF00BF0D48FFF74CF9D7
:101A300001280AD10A48FFF760F9012805D100BF43
:101A4000C01E0749086100BF00BF00BFFFF76CF868
:101A500000BF04480068401C0249086000BF10BD78
:101A6000002C01405800002010B52D48FFF72CF93C
:101A7000012853D100BF2A48FFF712F901280AD1E3
:101A80002748FFF726F9012805D100BF001F244988
:101A9000086100BF00BF2248FFF707F901280AD1FB
:101AA0001F48FFF71BF9012805D100BF801F1C4903
:101AB000086100BF00BF1A48FFF7FCF801280BD1EE
:101AC0001748FFF710F9012806D100BF6FF0080092
:101AD0001349086100BF00BF1148FFF7F0F8012863
:101AE0000BD10F48FFF704F9012806D100BF6FF0B2
:101AF00010000B49086100BF00BF0948FFF7E4F878
:101B000001280AD10648FFF7F8F8012805D100BFDF
:101B1000C01E0349086100BF00BF00BF10BD000028
:101B20000004004010B50248006802F07FFC10BDC0
:101B30005C00002000BFFEE70FB47CB50C0009ADCF
:101B400001D0611E00E00021CDE90001064B6A468C
:101B50002946089800F020F9002C02D0009A0021B4
:101B600011707CBC5DF814FB4D230008002809DBD4
:101B700000F01F02012191404209920002F1E0228F
:101B8000C2F800117047002809DB00F01F02012194
:101B900091404209920002F1E022C2F80011704720
:101BA00002480068C0F30220704700000CED00E01E
:101BB00002480068C0F30220704700000CED00E00E
:101BC00010B5002804DB0A07130E054A135406E07B
:101BD0000A07140E034A00F00F031B1FD45410BD54
:101BE00000E400E018ED00E010B5002804DB0A076F
:101BF000130E054A135406E00A07140E034A00F0B8
:101C00000F031B1FD45410BD00E400E018ED00E0EA
:101C100002E008C8121F08C1002AFAD170477047B5
:101C2000002001E001C1121F002AFBD17047000013
:101C30002DE9F04704460D4690461F46DDE9086948
:101C40000CB1012100E0002108468821FEF780FD4B
:101C50000DB1012100E0002108468921FEF778FD41
:101C6000A16D09B1012100E0002108468A21FEF79B
:101C70006FFD6567C4F87880E667012084F880000E
:101C800084F881000FB1C4F88470B9F1000F01D05D
:101C9000C4F88890A16D01F10C0000BF711E114ABB
:101CA000515C2944886000BF00BF0120686000BF0C
:101CB00000BF0220686000BF00BF701E1146085CB4
:101CC000285840F00201701E105C295000BFA06D22
:101CD000416841F00201416000BFA06DFEF74CFF7A
:101CE000BDE8F087F6470008014601F1100000E06A
:101CF000001D02681AB9024A12689042F8D3704770
:101D00003400002070B504460D460CB1012100E0FE
:101D1000002108467E21FEF71BFD0DB1012100E0E8
:101D2000002108467F21FEF713FD002084F85C00A7
:101D3000A5652846FEF720FF70BD000010B50648D7
:101D4000046803E02046FFF7CFFF0446034800681D
:101D50008442F7D310BD0000300000203400002082
:101D600010B504462146002001F018F810BD10B54A
:101D700001E000F8011B131EA2F10104A2B2F8D188
:101D800010BD10B501E000F8011B131EA2F1010403
:101D9000A2B2F8D110BD00002DE9FF4F8DB00F4663
:101DA0000546002606E025280BD0DDE90F129047F6
:101DB0006D1C761C28780028F5D111B03046BDE89E
:101DC000F08F0024A246A1460122E94900E0044325
:101DD00015F8013F203B02FA03F00842F7D12878BA
:101DE0002A2810D06FF02F022878A0F1300109299D
:101DF00014D80AEB8A0102EB410144F0020400EB23
:101E0000010A6D1CF0E701CF5FEA000A03D544F434
:101E10000054CAF1000A44F002046D1C28782E28F0
:101E200017D115F8010F44F004042A280ED06FF0E2
:101E30002F022878A0F1300109290AD809EB89017D
:101E400002EB410100EB01096D1CF2E757F8049B1E
:101E50006D1C28786C280FD006DC4C2817D0682819
:101E60000DD06A2814D104E0742810D07A280FD13C
:101E70000DE044F400140AE044F4801401E044F45A
:101E800040146978814202D104F580146D1C6D1CE8
:101E900028786E281ED00CDC632830D004DC0028A3
:101EA0008BD0582811D19FE0642867D069280CD1C5
:101EB00064E073282DD004DC6F2872D0702804D120
:101EC00094E075286ED078286DD0DDE90F12904728
:101ED000761C4BE1C4F30250022806D0032809D037
:101EE000042801CF09D0066040E101CFF117C0E915
:101EF00000613BE101CF068038E1067036E117F85A
:101F0000040B8DF8000000208DF80100EB46012045
:101F100003E057F804BB4FF0FF3061074FF00001BA
:101F200002D40DE008F10101884649450FDA8045E9
:101F3000F8DB1BF808100029F4D108E008F10101D2
:101F400088468142FADB1BF808100029F6D1DDE94A
:101F50000F23AAEB08008146214600F031F93044F6
:101F600000EB080604E0DDE90F121BF8010B9047B7
:101F7000B8F10108F7D221464846F2E00A21C4F33D
:101F800002524FF0000B0891022A04D001CFC11772
:101F9000032A09D00AE0FF1D27F00707F7E802012E
:101FA00008E02CE01EE01FE000B2C117042A01D1B6
:101FB00040B2C117021E71F1000206DA0023D0EB15
:101FC000030063EB01012D2202E0220504D52B2240
:101FD0008DF82420012203E0E20701D02022F7E758
:101FE000904653E00A210BE0102109E010214FF048
:101FF000000B44F004044FF00809089103E00821A5
:102000004FF0000B0891C4F30252022A04D001CF12
:102010000021032A06D006E0FF1D27F00707F7E896
:10202000020103E080B2042A00D1C0B24FF00008E0
:1020300022072BD52A78702A07D0DDF820C08CF033
:10204000100C5CEA0B0C05D00EE040228DF8242029
:10205000012208E050EA010306D030238DF8243035
:102060008DF8252002229046089B83F0080353EA4E
:102070000B030BD150EA010201D1620706D53022D1
:102080008DF824204FF00108A9F101092A78582A77
:1020900004D038A20B9208AA0A920BE03AA2F9E700
:1020A0005B46089AFEF74AFA0B9B9B5C0A9A521E03
:1020B0000A92137050EA0102F2D10A98ADEB0000C7
:1020C00000F1200B600702D524F4803401E04FF0CA
:1020D0000109D94502DDA9EB0B0000E0002000EB6F
:1020E0000B0141440890AAEB010AE00306D4DDE9A4
:1020F0000F232146504600F063F806444FF00009D4
:1021000008E009A911F80900DDE90F12904709F16B
:102110000109761CC145F4DBE0030CD5DDE90F2392
:102120002146504600F04CF8064404E0DDE90F1269
:1021300030209047761C0899481E08900029F5DC4D
:1021400008E00A980A990078491C0A91DDE90F1203
:102150009047761CBBF10001ABF1010BF1DC21468D
:102160005046DDE90F2300F019F806446D1C21E606
:10217000092801003031323334353637383961625D
:102180006364656600000000303132333435363721
:102190003839414243444546000000002DE9F041F2
:1021A000044600251E461746880404D405E0394637
:1021B0002020B0476D1C641EF9D52846BDE8F0818B
:1021C0002DE9F041044600251E469046C80301D57E
:1021D000302700E02027880404D505E04146384632
:1021E000B0476D1C641EF9D52846BDE8F0810FB4D8
:1021F000DDE900108A68C0F30F231A40C0F30F23F3
:102200009A4201D1012200E00022D0B204B070470E
:102210007CB504460CB1012100E000210846CF2125
:10222000FEF796FAA169D1E90401CDE90001A5699B
:102230006E6995E80F00B0477CBD2DE9F047074671
:10224000884614461D464FF000090FB1012100E0F9
:1022500000210846FA21FEF77BFA0CB1012100E0CB
:1022600000210846FB21FEF773FA0DB1012100E0C1
:1022700000210846FC21FEF76BFA384600F05BFEB1
:102280004146384600F045FF8146002606E0FF2122
:10229000384600F03EFFA055701CC6B2AE42F6DBD9
:1022A000384600F02DFE4846BDE8F0872DE9FC4198
:1022B00004462169D1E90401CDE900012669F768E6
:1022C0003B4696E80700B84794F860102046226B1A
:1022D00090476620015D2046226B904705462169A4
:1022E000D1E90401CDE900012669D6E902733A4635
:1022F000D6E90001B8472846BDE8FC8170B5044620
:10230000002508E02846691C8DB244F62061884209
:1023100000DD07E000BF2046FFF7C8FF00F0010026
:102320000028EFD100BF70BD0FB4DDE90001C1F39B
:102330000F22426100BF04B070470FB4DDE9000115
:10234000C1F30F22026100BF04B070474A68002A3F
:1023500006D00A68531C0B6010704868401E486025
:10236000704710B504460CB1012100E00021084679
:10237000A321FEF7EDF9D4F8880018B12046D4F86F
:1023800088108847D4F8840018B12046D4F8841007
:10239000884710BDF0B50346002083F88100DC6F4C
:1023A000586F661E224FBE5D865926F00107661ED5
:1023B000DFF87CC01CF80660875100BFDC6F586FE7
:1023C000661E6746BE5D0644F16000BFDC6F586F55
:1023D000661EBE5D064476686FF30F061643671EE1
:1023E0001CF8077007447E6000BFDC6F586F661EE4
:1023F0006746BE5D865946F00107661E1CF80660FA
:10240000875100BF002507E0681C85B24CF25030B0
:10241000854201DD00BF03E093F881000028F3D07E
:1024200000BF93F88100012800D1F0BD0020FCE737
:10243000F647000870B504460D4600260CB1012190
:1024400000E00021084640F22911FEF781F92046FC
:1024500000F071FD2946204600F05BFE0021204679
:1024600000F057FE0646204600F04AFD304670BD9B
:102470002DE9FC4105460E4600270DB1012100E083
:102480000021084640F23D11FEF762F92C460CB1DE
:10249000012100E00021084640F2E521FEF758F94D
:1024A000A169D1E90401CDE90001D4F818C0DCF834
:1024B0000C8043469CE80700C04700BF284600F058
:1024C0003AFD3146284600F024FE0746284600F033
:1024D00017FD3846BDE8FC812DE9FC4705460E4650
:1024E00017464FF000080DB1012100E00021084619
:1024F0004FF4A871FEF72CF92C460CB1012100E035
:102500000021084640F2DA21FEF722F9A169D1E95B
:102510000401CDE90001D4F818C0DCE902934A4671
:10252000DCE90001C84700BF284600F004FD002494
:1025300007E03178284600F0ECFD8046761C601CF0
:1025400084B2BC42F5DB284600F0DAFC4046BDE828
:10255000FC872DE9F04104460E46154600270CB1D4
:10256000012100E0002108464FF48A71FEF7F0F8DF
:10257000204600F0E0FC3146204600F0CAFD074648
:102580002946204600F0C5FD204600F0B9FC38463B
:10259000BDE8F0810FB430B5DDE90301C268C1F3D5
:1025A0000F2323EA020402EA030544EA0544046116
:1025B00000BF30BC5DF814FB7CB504462169D1E94D
:1025C0000401CDE900012569EE68334695E807006E
:1025D000B0476320015D2046226B90472169D1E915
:1025E0000401CDE900012569D5E902633246D5E948
:1025F0000001B0477CBD7CB504462169D1E90401E6
:10260000CDE900012569EE68334695E80700B0473B
:102610006220015D2046226B90472169D1E90401C7
:10262000CDE900012569D5E902633246D5E900010B
:10263000B0477CBD2DE9F04106460F4614461D46C5
:102640004FF000080EB1012100E000210846DE2114
:10265000FEF77EF80CB1012100E000210846DF21E1
:10266000FEF776F80DB1012100E000210846E021D7
:10267000FEF76EF8304600F05EFC3946304600F05A
:1026800048FD804604E02178304600F042FD641C9D
:10269000281EA5F10101CDB2F5D1304600F030FC85
:1026A0004046BDE8F081000010B515A1032001F0FF
:1026B000A1F8C82000F0BAF800F09EFF002405E061
:1026C000204601F03DF804F10A00C4B2642CF7DDA5
:1026D00000200E4908600E49086000BF0D48FEF753
:1026E00093FA0C48FEF795FA00BF00BF0A48FEF7C0
:1026F0008BFA0948FEF78DFA00BF00F076FF10BD97
:102700004C4F4144494E472E2E2E0000040000201D
:102710000C000020002C01400004004010B50348CC
:1027200000F054F8024800F0DBF910BD040000206E
:102730000C00002000B587B001F048FE01F0EDFA72
:1027400040F608011E48FEF7CCF941F21000010ADC
:102750001B4A116100BF01111A48FEF7C2F940F28D
:1027600002211848FEF7BDF9642000F05FF841F23D
:102770001001134800F09EF8049048F280011048C0
:1027800000F098F8019042F220010D4800F092F814
:10279000039044F240010A4800F08CF802900021B6
:1027A000084600F087F805900021084600F082F8FE
:1027B000069001AA0449002001F098FB07B000BD73
:1027C00000080140000C01400030014038B50446CB
:1027D00000200090206810B1122819D10EE000BF2F
:1027E000002001F037FB002001F0AEFB00BF0B48DA
:1027F0000068606000BF1220206000BF0749606869
:102800000968081A642801D2002038BD00BFE7E734
:102810000020206000900320F7E70000580000200F
:1028200001490860704700001C00002070B5044694
:102830001E2094FBF0F594FBF0F100FB114604E040
:1028400047F2305000F012F86D1E002DF8D12EB175
:102850004FF47A7106FB01F000F008F870BD00E05B
:1028600000BF011EA0F10100FAD1704770B5034608
:1028700000224FF0E02675690D4E366803FB06F422
:102880004FF0E026B16910E04FF0E026B0698842D1
:102890000BD0884202D20E1A324402E02E1A0E44A5
:1028A00032440146A24200D300E0EDE700BF70BD14
:1028B0001C0000202DE9F04105460E461827394638
:1028C000002000F06BFA04460CB1012100E0002169
:1028D00008463621FDF73CFF256066600548A0608C
:1028E0000548E06005482061054860612046BDE874
:1028F000F08100003B2300082923000895250008EB
:10290000EF21000810B500BF01220E490E48FEF766
:10291000F4F800BF0B490C48FEF7EBF80B490A48E6
:10292000FEF7E7F80420FFF7A1FF06490648FEF787
:10293000DCF80420FFF79AFF04490348FEF7D5F8B6
:1029400010BD000010001004000C01402000200405
:1029500010B500BF01220E490E48FEF7CEF800BFA9
:102960000D490C48FEF7C1F809490A48FEF7BDF8C1
:102970000420FFF77BFF08490648FEF7BAF8044930
:102980000448FEF7B6F80420FFF770FF10BD000002
:1029900010001004000C01402000200410B5002499
:1029A000082213491348FEF7A8F811491148FEF709
:1029B000A0F80420FFF75AFF0F490E48FEF799F8D8
:1029C0000420FFF753FF07E0601CC4B2FA2C03DDBC
:1029D000FFF7BEFF002010BD05490648FEF770F85E
:1029E0000028F1D104490348FEF77FF80120F2E7FF
:1029F00010001004000C01402000200470B50446B3
:102A0000002500BF012217491748FEF776F800BFDE
:102A100016491548FEF769F800BF1FE0E00920B12C
:102A200010491148FEF765F803E00E490E48FEF71D
:102A30005CF86006040E0220FFF718FF0B490A48F5
:102A4000FEF757F80220FFF711FF08490648FEF786
:102A50004CF80220FFF70AFF681CC5B2082DDDDB29
:102A600070BD000010001004000C01402000200484
:102A700038B5044600208DF800008DF80140FFF7BE
:102A800041FF7820FFF7BAFFFFF788FF9DF80000AD
:102A9000FFF7B4FFFFF782FF9DF80100FFF7AEFFDD
:102AA000FFF77CFFFFF754FF38BD38B504464020E0
:102AB0008DF800008DF80140FFF724FF7820FFF724
:102AC0009DFFFFF76BFF9DF80000FFF797FFFFF7F3
:102AD00065FF9DF80100FFF791FFFFF75FFF38BD2D
:102AE000F8B5044600200090206810B12B284AD188
:102AF0003FE000BF2648274BD968C0F30F2222EAE7
:102B0000010301EA020543EA0543224D2B6100BFA0
:102B100021A20221002001F077F821490868096804
:102B2000491C1F4B1960FDF790FC054600232A46FF
:102B30000221282000F074FE1AA20421002001F0D6
:102B400063F8002001F0BEF946683046FDF774FCDA
:102B5000054600232A460421282000F061FE01F0EA
:102B600031F900BF11480068606000BF2B20206071
:102B700000BF0E4960680968081A642801D2002065
:102B8000F8BD00BFB6E70020206000900320F7E703
:102B90002000200400100140207469636B3A00009B
:102BA00018000020206366673A00000058000020EB
:102BB00008B50120284989690143274A91611146D6
:102BC00089690140009100BF00BF00071146C96933
:102BD0000143D1611146C9690140009100BF00BFA6
:102BE000032002461D4B19684FF6FF0319401C4B8A
:102BF0000B4343EA0221194B196000BF00BF19487B
:102C0000406820F0E06040F000701649486000BF66
:102C1000FEF748FE144800681449B0FBF1F084B296
:102C20002046FFF7FDFDFEF7F7F9FEF7C7F9FEF7BF
:102C300003FBFEF799FBFEF7C5FAFEF75DFBFEF717
:102C40007BFA002000F014F8FFF774FDFFF72CFD6D
:102C500001E0FFF763FDFCE7001002400CED00E02F
:102C60000000FA05000001400000002040420F0073
:102C700010B504460C4951F824104A000B4951F88C
:102C80002400002100F09EF8094951F8242007494A
:102C9000083951F82400002100F094F8012103487C
:102CA0000830015510BD0000384800084C000020D5
:102CB000484800082DE9F04704460F460025A9467C
:102CC0002348005D20B9224818380168204688470B
:102CD0001FB94FF0FF30BDE8F0871E4850F82400C0
:102CE000B7FBF0F61B4850F82400B7FBF0F100FBEF
:102CF000117000B1761C184850F82400451E22E0DF
:102D00001348083850F8240030F8150010B909F1BC
:102D1000010901E04FF00009B14513D14FF000085F
:102D200009E00B48083850F8240005EB080220F8A9
:102D3000126008F10108B045F3D3064850F82400AA
:102D40006843C8E76D1E002DDADA4FF0FF30C2E7A6
:102D500054000020404800083848000810B50146DB
:102D60000023002207E00B4850F8210030F8120041
:102D700000B15B1C521C084850F821009042F2D868
:102D800064205843044C54F82140B0FBF4F0C0B226
:102D900010BD00004C0000203848000870B5044603
:102DA0000E4631462046FFF785FF0546681C08B9E8
:102DB000002070BD024850F824002844F9E70000C4
:102DC0004400002030B5034601E003F8011B141E47
:102DD000A2F10102F9D130BD0FB42DE9F041054651
:102DE0000D9F022D01DA012100E000210846382163
:102DF000FDF7AEFC902631460020FFF7CFFF0446DA
:102E000000BF201D07A9182203E011F8013B00F8BC
:102E1000013B131EA2F10106B2B2F6D100BF6780DA
:102E20002570012084F85C002449A1642449E164F0
:102E30002449616524492165002D2ED12348E06194
:102E4000234921622349A1622349E1622349616246
:102E500023492163234961632349E1632349A16332
:102E60002349216423496164052084F8600001211D
:102E7000612001550621622001550421632001557E
:102E8000032164200155022165200155A5216620FA
:102E900001550021712001550AE0012D04D1164889
:102EA000E0611649216203E061210020FDF750FC3A
:102EB0002046BDE8F0015DF814FB0000051D000888
:102EC000311C0008952300086323000853250008DF
:102ED00035240008352600083B220008112200088E
:102EE00013310008BF320008992F0008A5330008ED
:102EF000B3350008C130000871240008D924000847
:102F00007CB504460CB1012100E0002108464FF4D5
:102F10003C71FDF71DFC2169D1E90401CDE90001F7
:102F20002569D5E902633246D5E90001B04720465C
:102F300000F01BF87CBD7CB504460CB1012100E01B
:102F4000002108464FF43F71FDF702FC2169D1E9E9
:102F50000401CDE900012569EE68334695E80700D4
:102F6000B047204600F001F87CBD70B5044600254E
:102F70000CB1012100E00021084640F26511FDF787
:102F8000E7FB6588002D06DD00E000BF281EA5F1E7
:102F900001018DB2F9D170BD2DE9FC4704460D4603
:102FA000174698464FF0010A00260CB1012100E0B7
:102FB000002108464FF42571FDF7CAFB0FB101212E
:102FC00000E00021084640F29521FDF7C1FBB8F171
:102FD000000F01DD012100E00021084640F29621AA
:102FE000FDF7B6FB2169D1E90401CDE90001D4F870
:102FF00010C0DCF80C904B469CE80700C8476420E2
:10300000015D2046226B9047064616B90020BDE8B8
:10301000FC876720005D022810D1C5F307212046F8
:10302000226B904706460EB90020F0E7E9B2204631
:10303000226B9047064626BB0020E8E76720005D2C
:10304000032819D1C5F307412046226B9047064655
:103050000EB90020DBE7C5F307212046226B90471D
:1030600006460EB90020D2E7E9B22046226B90470F
:10307000064636B90020CAE740F2BF210020FDF71E
:1030800067FB4FF000090AE06620015D2046226BD5
:10309000904707F8090009F101001FFA80F9C145BE
:1030A000F2DB2169D1E90401CDE90001D4F810C0B7
:1030B000DCE902934A46DCE90001C8475046A6E72E
:1030C0002DE9FC4104460D462169D1E90401CDE911
:1030D00000012769D7F80CC0634697E80700E0476E
:1030E00029462046226B90476620015D2046226BD0
:1030F000904706462169D1E90401CDE9000127691D
:10310000D7E902C36246D7E90001E0473046BDE88F
:10311000FC812DE9FC4704460D464FF0FF080CB139
:10312000012100E00021084640F2B111FDF710FB3B
:1031300094F85C0001287CD1002795E026460EB16A
:10314000012100E00021084640F22931FDF700FB93
:10315000F168D1E90401CDE90001D6F80CC0DCF832
:103160000C904B469CE80700C84700BF2046FFF77D
:10317000FCFE05F08000C0B126460EB1012100E042
:10318000002108464FF44271FDF7E2FA7168D1E977
:103190000401CDE90001D6F804C0DCE902934A46F7
:1031A000DCE90001C84700BF18E026460EB1012146
:1031B00000E00021084640F21331FDF7C9FA7168BA
:1031C000D1E90401CDE90001D6F804C0DCF80C9087
:1031D0004B469CE80700C84700BF00BF2046FFF7EA
:1031E000C4FE26460EB1012100E00021084640F24F
:1031F0001E31FDF7ADFAF168D1E90401CDE9000116
:10320000D6F80CC0DCE902934A46DCE90001C84765
:1032100000BF2046FFF7A9FE6806050E4FEA48608A
:103220004FEA1068A0680068E0B1264616B1012197
:1032300001E01FE0002108464FF44D71FDF788FAC8
:10324000B168D1E90401CDE90001D6F808C0DCF885
:1032500014909CE80F00C847012803D108F1010031
:1032600000F0FF08781CC7B2082FFFF667AF404692
:10327000BDE8FC87A06D00F10C010D7000BF4FF0A0
:10328000FF320221204600F043F808B9FF20EFE7A3
:103290004FF0FF320121204600F03AF808B9FF2034
:1032A000E6E74FF0FF320221204600F031F808B97E
:1032B000FF20DDE7A06D017B88464046D8E77CB55E
:1032C00004460CB1012100E0002108464FF433719F
:1032D000FDF73EFA2169D1E90401CDE90001256934
:1032E000EE68334695E80700B0470A20FFF7B7FAC3
:1032F0002169D1E90401CDE900012569D5E902631D
:103300003246D5E90001B0470A20FFF7A8FA7CBD94
:103310002DE9F04104460D46164600270CB1012167
:1033200000E00021084640F27311FDF711FA022D6A
:103330000FD107E038467F1CB04202D90020BDE81B
:10334000F08100BFA06D8168C1F340010029F1D078
:1033500026E0012D0ED106E038467F1CB04201D98F
:103360000020ECE700BFA06D816801F00101002999
:10337000F2D015E0802D0ED106E038467F1CB04219
:1033800001D90020DBE700BFA06D8168C1F3C01147
:103390000029F2D004E04FF4D0710020FDF7D8F9F5
:1033A0000120CCE72DE9FC5F04460D461746984600
:1033B0004FF0010A00260CB1012100E0002108466F
:1033C00040F20D21FDF7C4F90FB1012100E0002109
:1033D000084640F20E21FDF7BBF9B8F1000F01DD00
:1033E000012100E00021084640F20F21FDF7B0F96D
:1033F000A16E09B1012100E0002108464FF40471DB
:10340000FDF7A6F9D4F868902046FFF7F4F8216993
:10341000D1E90401CDE90001D4F810C0DCF80CB00A
:103420005B469CE80700D8476520015D2046226B7B
:103430009047064616B90020BDE8FC9F6720005D56
:10344000022810D1C5F307212046226B904706467B
:103450000EB90020F0E7E9B22046226B90470646FD
:10346000DEB90020E8E7C5F307412046226B90470C
:1034700006460EB90020DFE7C5F307212046226B80
:10348000904706460EB90020D6E7E9B22046226BE7
:10349000904706460EB90020CEE76EE03978204608
:1034A000226B904706460EB90020C5E77F1C7120AD
:1034B000005D002861D16D1CB5FBF9F009FB1050CF
:1034C00000285AD1B8F1000F57DD2169D1E9040174
:1034D000CDE90001D4F810C0DCE902B35A46DCE9BA
:1034E0000001D8472046FEF709FF2046FFF783F882
:1034F0002169D1E90401CDE90001D4F810C0DCF85C
:103500000CB05B469CE80700D8476520015D20466B
:10351000226B904706460EB900208DE76720005DBC
:10352000022810D1C5F307212046226B904706469A
:103530000EB9002080E7E9B22046226B904706468C
:10354000DEB9002078E7C5F307412046226B90479B
:1035500006460EB900206FE7C5F307212046226B0F
:10356000904706460EB9002066E7E9B22046226B76
:10357000904706460EB900205EE7B8F10000A8F1BA
:1035800001011FFA81F889D12169D1E90401CDE94E
:103590000001D4F810C0DCE902B35A46DCE90001AE
:1035A000D8472046FEF7AAFE2046FFF705F850460A
:1035B00042E770B504460D4616460CB1012100E005
:1035C0000021084640F27F21FDF7C2F82046FFF7B0
:1035D00012F8324629462046E36998472046FEF70E
:1035E0008DFE2046FEF7E8FF70BD10B500F004F830
:1035F00000F0E8FB10BD000010B54FF48062002120
:103600000448FEF7BEFB4FF48062FF210248FEF73C
:10361000B8FB10BD80280020802C00202DE9FC4F35
:1036200004460D4616461F46301B01D5A01B00E080
:10363000301B8146781B01D5E81B00E0781B8246D1
:10364000B44201DA012001E04FF0FF300190BD42A9
:1036500001DA012001E04FF0FF300090A9EB0A00F1
:103660000FFA80F821E0294620460B9A00F022F854
:10367000B44202D1BD4200D118E04FEA48000FFA2F
:1036800080FBCAF10000834506DDA8EB0A000FFAB3
:1036900080F801982044C4B2CB4506DA08EB090053
:1036A0000FFA80F800982844C5B2DCE700BFBDE8F7
:1036B000FC8F0000F0B503461446802B01DA402948
:1036C00000DBF0BD012C1CD1CD1701EB5575ED10C1
:1036D00003EBC515194E755D0A46CE1701EB5676FC
:1036E000F610A1EBC6070126BE403543EEB20846F0
:1036F000CD1701EB5575ED1003EBC5150F4F7E553A
:103700001AE0CD1701EB5575ED1003EBC5150B4E07
:10371000755D0A46CE1701EB5676F610A1EBC6078B
:103720000126BE40B5430846CE1701EB5676F6108B
:1037300003EBC616014FBD5500BFC2E7802800202D
:103740003EB504460A25012005F118010A236C2222
:103750000090184600F01CF801200090201DC2B215
:1037600005F11A0107230C2000F0BCFA234606A23B
:10377000052101A8FEF7E0F901AA02212C2000F0A2
:1037800071FA00F01FFB3EBD2533642525000000C3
:103790002DE9F84104460D4616461F46DDF81C800B
:1037A000A019C2B22B4629462046CDF80080FFF76B
:1037B00035FFE819C3B2A019C2B2E819C1B2204658
:1037C000CDF80080FFF72AFFE819C3B22246294648
:1037D0002046CDF80080FFF721FFE919CBB2A119EF
:1037E000CAB2A119C8B22946CDF80080FFF716FF6A
:1037F000BDE8F88170B505460C462046FCF7A6FCEE
:1038000000EB40008021A1EB4000C0F347062246B8
:103810002946304600F0F8F900F0D4FA70BD0000F7
:103820002DE9F04F87B005460E4691469A46002096
:10383000039004900590029000248346002148469E
:10384000FCF768FE07D22D222046611CCCB203A9EA
:103850000A5489F00049E3494846FCF765FE02D264
:1038600007B0BDE8F08FC4F10800C0B20290DE4995
:103870004846FCF759FE59D8DB494846FCF7F7FCA7
:103880008046DA49FCF769FC0746FCF7FCFDC2B24A
:103890002046611CCCB203A90A544846FCF7DAFD65
:1038A00042F2107190FBF1F201FB12004FF47A71B9
:1038B00090FBF1F03030C2B22046611CCCB203A9BB
:1038C0000A544846FCF7C6FD4FF47A7190FBF1F2BA
:1038D00001FB1200642190FBF1F03030C2B22046AF
:1038E000611CCCB203A90A544846FCF7B3FD64211D
:1038F00090FBF1F201FB12000A2190FBF1F0303055
:10390000C2B22046611CCCB203A90A544846FCF757
:10391000A1FD0A2190FBF1F201FB12003030C2B28E
:103920002046611CCCB203A90A54C2E0B049484603
:10393000FCF7FAFD48D84846FCF78CFD42F21071BE
:1039400090FBF1F201FB12004FF47A7190FBF1F061
:103950003030C2B22046611CCCB203A90A5448469A
:10396000FCF778FD4FF47A7190FBF1F201FB120045
:10397000642190FBF1F03030C2B22046611CCCB221
:1039800003A90A544846FCF765FD642190FBF1F257
:1039900001FB12000A2190FBF1F03030C2B2204648
:1039A000611CCCB203A90A544846FCF753FD0A2116
:1039B00090FBF1F201FB12003030C2B22046611CD4
:1039C000CCB203A90A5474E08A494846FCF7ACFD1E
:1039D00034D84846FCF73EFD4FF47A7190FBF1F283
:1039E00001FB1200642190FBF1F03030C2B220469E
:1039F000611CCCB203A90A544846FCF72BFD642194
:103A000090FBF1F201FB12000A2190FBF1F0303043
:103A1000C2B22046611CCCB203A90A544846FCF746
:103A200019FD0A2190FBF1F201FB12003030C2B205
:103A30002046611CCCB203A90A543AE06E494846BC
:103A4000FCF772FD21D84846FCF704FD642190FB89
:103A5000F1F201FB12000A2190FBF1F03030C2B20A
:103A60002046611CCCB203A90A544846FCF7F2FC7C
:103A70000A2190FBF1F201FB12003030C2B2204665
:103A8000611CCCB203A90A5413E000214846FCF79C
:103A90004BFD0ED84846FCF7DDFC0A2190FBF1F205
:103AA00001FB12003030C2B22046611CCCB203A927
:103AB0000A54BAF1000F6ADD072C68DA2E2220467C
:103AC000611CCCB203A90A544846FCF7C3FC8046EB
:103AD000FCF7B2FC07464946FCF794FB8146BAF175
:103AE000010F1ED1082C1CDA43494846FCF78DFB18
:103AF00081464846FCF7FAFC0022404BCDE9000124
:103B0000FCF7F3FB0746FCF7D2FC0A2190FBF1F22D
:103B100001FB12003030C2B22046611CCCB203A9B6
:103B20000A54BAF1020F32DB082C30DA3149484628
:103B3000FCF76BFB81464846FCF78CFC642190FB4C
:103B4000F1F201FB12000A2190FBF1F03030C2B219
:103B50002046611CCCB203A90A54082C17DA484647
:103B6000FCF7C4FC0022254BCDE90001FCF7BDFBAE
:103B70000746FCF79CFC0A2190FBF1F201FB1200C6
:103B80003030C2B22046611CCCB203A90A5422E0F4
:103B900003A810F80B002038C0B20290782D02DD87
:103BA0000025701CC6B200240DE0029800EB400016
:103BB000134901EB4000005D05EBC6112144114A99
:103BC0005054601CC4B2062CEFDBA81DC5B20BF12B
:103BD000010000F0FF0B03A810F80B000028D7D15C
:103BE00000BF3DE60000FA4600401C46000040428F
:103BF00000007A440000C842000020410000E03F7D
:103C00007A48000880280020F0B5134600250022DD
:103C100000241EE01E5D203EF5B27E2802DD00205D
:103C20004E1CF1B200220EE005EB45060B4F07EBF0
:103C30004606B65C00EBC1171744DFF824C00CF849
:103C40000760561CF2B2062AEEDB861DF0B2661C37
:103C5000F4B21E5D002EDDD1F0BD00007A480008F0
:103C600080280020F0B503461446002200200025DD
:103C700030E0665D203EF2B2782B02DD00234E1C60
:103C8000F1B200200CE000EB0216144FBE5D03EB16
:103C9000C1170744DFF848C00CF80760461CF0B2B3
:103CA0000828F0DB00200EE000EB021608360B4F70
:103CB000BF5D4E1C03EBC6160644DFF824C00CF8AB
:103CC0000670461CF0B20828EEDB03F10806F3B2DA
:103CD0006E1CF5B2665D002ECBD1F0BDA24A000885
:103CE000802800202DE9F84306460D4617469846E1
:103CF000DDF8209000240CE02819C3B2F019C2B2FC
:103D00002819C1B23046CDF80090FFF787FC601C3F
:103D1000C4B24445F0DBBDE8F88310B5AE20FEF731
:103D2000A7FE2020FEF7A4FE1020FEF7A1FEC8206B
:103D3000FEF79EFE0020FEF79BFE1020FEF798FE89
:103D40004020FEF795FE8120FEF792FEFF20FEF751
:103D50008FFEA120FEF78CFEA620FEF789FEA8208C
:103D6000FEF786FE3F20FEF783FEA420FEF780FECE
:103D7000D320FEF77DFE0020FEF77AFED520FEF769
:103D800077FEF020FEF774FED920FEF771FE2220A8
:103D9000FEF76EFEDA20FEF76BFE1220FEF768FEDD
:103DA000DB20FEF765FE2020FEF762FE8D20FEF789
:103DB0005FFE1420FEF75CFEAF20FEF759FEFFF712
:103DC00014FC10BD70B500242DE0002600200DE08D
:103DD00000EBC4111D4A515C00EBC4121C4B9A5CF1
:103DE000914201D0012603E0411CC8B28028EFDBDC
:103DF00000BFB6B104F1B001C8B2FEF739FE012030
:103E0000FEF736FE1020FEF733FE002507E005EB37
:103E1000C4110E4A505CFEF748FE681CC5B2802DE6
:103E2000F5DB601CC4B2082CCFDB094807494FF40E
:103E3000806203E011F8013B00F8013B131EA2F180
:103E40000104A2B2F6D100BF70BD0000802800209E
:103E5000802C00207FB5044680208DF808000020CB
:103E60008DF809008DF80A008DF80B0002208DF8FE
:103E70000C0002A9204600F005F902A80021052245
:103E800001E000F8011B131EA2F10105AAB2F8D14E
:103E900000BF6420FEF7CAFC0020009001908DF85E
:103EA00008006A4602A9204600F082F89DF8040046
:103EB00004EB4401024A02EB810148607FBD00002F
:103EC0008030002010B50446012C01DA012100E009
:103ED000002108463421FCF73BFC04EB4400024976
:103EE00001EB800010BD0000803000202DE9FF4173
:103EF00004460F461546012C01DA012100E000219D
:103F000008462B21FCF724FC04EB44000D4901EB8F
:103F1000800600200390D5E90412E8688DE80700C8
:103F2000002095E80E00FEF757FF3060316809B1B8
:103F3000012100E0002108462F21FCF709FCBDE823
:103F4000FF810000803000207FB50546012D01DA99
:103F5000012100E0002108464C21FCF7F9FB05EBAC
:103F60004500124901EB800600200290039000906A
:103F7000019021208DF808006A4602A9284600F029
:103F800017F800249DF80100044324029DF8020064
:103F9000044324029DF80300044324029DF8040016
:103FA0000443B460204604B070BD0000803000209F
:103FB0002DE9FC4106460F469046012E01DA01210B
:103FC00000E0002108461321FCF7C2FB06EB460087
:103FD0002B4901EB800420680169D1E90401CDE996
:103FE000000120680569D5F80CC0634695E8070014
:103FF000E047002507E0795D2068026B904708F8EC
:104000000500681C85B2052DF5DB20680169D1E942
:104010000401CDE9000120680569D5E902C36246C3
:10402000D5E90001E04700BF00BF00BF206801697B
:10403000D1E90401CDE9000120680569D5F80CC07B
:10404000634695E80700E047002507E0795D2068B2
:10405000026B904708F80500681C85B2052DF5DB5A
:1040600020680169D1E90401CDE9000120680569F2
:10407000D5E902C36246D5E90001E047BDE8FC810D
:10408000803000202DE9FC4105460F46012D01DA64
:10409000012100E0002108460721FCF759FB05EB50
:1040A0004500154901EB800420680169D1E904014C
:1040B000CDE9000120680669D6F80CC0634696E891
:1040C0000700E047002605E0B95D2068026B9047D5
:1040D000701C86B2052EF7DB20680169D1E9040166
:1040E000CDE9000120680669D6E902C36246D6E937
:1040F0000001E047BDE8FC818030002010B5044697
:1041000004B910BD00202085A07D012808D1606A77
:1041100030B1218C89040A0C0021606AFDF727FE6A
:1041200000BFEEE72DE9F05F064688461546994642
:10413000DDE90B7BDDF828A00EB1012100E00021B4
:1041400008462921FCF704FB4420FDF709FE04463C
:104150000CB1012100E0002108462C21FCF7F8FAFF
:104160000120E07500202076C4F83C902584C4F836
:1041700040B0A786002D0CDD2846FDF7F1FDE0617B
:10418000E16909B1012100E0002108463E21FCF768
:10419000DFFA002F0CDD3846FDF7E2FD2063216BCE
:1041A00009B1012100E0002108464521FCF7D0FAC1
:1041B00084F8158084F82CA066602046BDE8F09F46
:1041C00010B5044604B910BD002060852046FFF7F5
:1041D00095FF00BFF7E710B504460CB1012100E0E0
:1041E0000021084640F2D711FCF7B2FA012084F80A
:1041F00038002169A068FCF70FFB2069082865D208
:10420000DFE800F06404111E2C3A485600BFA06895
:104210000168C1F3400121B1A0680221416000BFE3
:1042200000BF00BF53E000BFA0680168C1F34011A8
:1042300021B1A0682021416000BF00BF00BF46E05F
:1042400000BFA0680168C1F3402129B1A0684FF404
:104250000071416000BF00BF00BF38E000BFA06830
:104260000168C1F3403129B1A0684FF400514160A9
:1042700000BF00BF00BF2AE000BFA0680168C1F313
:10428000404129B1A0684FF40031416000BF00BF38
:1042900000BF1CE000BFA0680168C1F3405129B114
:1042A000A0684FF40011416000BF00BF00BF0EE0E6
:1042B00000BFA0680168C1F3406129B1A0684FF058
:1042C0000071416000BF00BF00BF00E000BF00BF41
:1042D000606800BF00BF00BF00F10C0252E8002F71
:1042E00042F0400100F10C0242E80013002BF3D130
:1042F00000BF00BF2069082865D2DFE800F0640431
:10430000111E2C3A485600BFA0680168C1F3C001D5
:1043100021B1A0680821416000BF00BF00BF53E089
:1043200000BFA0680168C1F3C01121B1A06880215D
:10433000416000BF00BF00BF46E000BFA068016849
:10434000C1F3C02129B1A0684FF40061416000BFF2
:1043500000BF00BF38E000BFA0680168C1F3C031F2
:1043600029B1A0684FF40041416000BF00BF00BF09
:104370002AE000BFA0680168C1F3C04129B1A0686C
:104380004FF40021416000BF00BF00BF1CE000BF30
:10439000A0680168C1F3C05129B1A0684FF40001C1
:1043A000416000BF00BF00BF0EE000BFA068016811
:1043B000C1F3C06129B1A0684FF00061416000BF46
:1043C00000BF00BF00E000BF00BF10BD0EB5134826
:1043D000006808BB0020F0210122114BCDE900212B
:1043E00002900A4601210F48FFF79CFE0B49086026
:1043F0000020096808700C48084909688860052091
:1044000006490968C8600420044909680861002158
:104410000248006800F0E2F80EBD00005C000020D9
:104420005F470008003801400000024038B50446EC
:1044300004B938BD6068C168C1F34011B9B16068A2
:104440000168C1F3401191B1608D218C884202DB7B
:104450002046FFF7B5FE61684A68D2B2608D411C04
:104460006185E1690A5400202076E0753FE06068CC
:10447000C168C1F30011002939D060680168C1F337
:104480000011002933D0607D01282BD1D4E902012D
:104490004A1E514B9A5C02445268208C801A6085F7
:1044A000207DF8B9D4E90201FCF7B6F9E06B80B1E0
:1044B000608D00280DDD608D218C884209DC628DC5
:1044C0002078E36BE1699847228C0021E069FDF7D1
:1044D0004EFC228CD4E90201FCF7D8F9D4E90201A0
:1044E000FCF7A8F9002060856068FCF7A8FC60680C
:1044F000C168C1F3801151B16068FCF706FD30B1AD
:10450000206C08B1206C80476068FCF7A0FCA07D9F
:1045100001285ED101256068C168C1F3002171B135
:104520006068016801F0010149B102256068016815
:10453000009100BF4168009100BF00BF00BF6068EC
:10454000FCF7D4FC68B16068FCF7D0FC48B10425E6
:1045500060680168009100BF4168009100BF00BF22
:1045600000BF6068FCF7C7FC60B16068FCF7C3FC83
:1045700040B160680168009100BF4168009100BFD0
:1045800000BF00BF6068FCF7BBFC68B16068FCF767
:10459000B7FC48B1102560680168009100BF416810
:1045A000009100BF00BF00BF012D11D0606A78B13B
:1045B000618D491E88B2228D616A01EB82014880BB
:1045C000228D616A01F82250218D491C218500BF8E
:1045D00000BF00BF2DE70000CC47000870B50446BF
:1045E0000D46607D90B9A575606800BF00BF00BF33
:1045F00000F10C0252E8002F42F0200100F10C0201
:1046000042E80013002BF3D100BF70E00020A0753A
:104610006068FCF714FC2169A068FCF7FDF8D4E998
:104620000201FCF7F9F86068011D0E463246D4E934
:104630000201FCF787F9E269D4E90201FCF748F9C5
:10464000228CD4E90201FCF721F9D4E90201FCF73C
:10465000FFF8D4E90201FCF7EDF8606800BF00BF85
:1046600000BF00F1140252E8002F42F0400100F1B7
:10467000140242E80013002BF3D100BF00BF6068B2
:1046800000BF00BF00BF00F10C0252E8002F42F053
:10469000100100F10C0242E80013002BF3D100BF1F
:1046A00000BF6068011D0E4632462169A068FCF714
:1046B00049F9226B2169A068FCF70AF92169A06811
:1046C000FCF7C6F8606800BF00BF00BF00F114022D
:1046D00052E8002F42F0800100F1140242E800137A
:1046E000002BF3D100BF00BF012084F83800A07D6B
:1046F000012833D1606A68B9218C8800FDF730FB4E
:104700006062616A09B1012100E00021084682214E
:10471000FCF71EF8606800BF00BF00BF00F10C028C
:1047200052E8002F42F4807100F10C0242E80013BD
:10473000002BF3D100BF00BF606800BF00BF00BF07
:1047400000F1140252E8002F42F0010100F11402BE
:1047500042E80013002BF3D100BF00BF70BD7047CB
:10476000081C3044586C8000000000040404000061
:10477000080000000800000800000008000204060D
:10478000080A0C00010203040506081C3044586C9A
:10479000800000000004040400000800000008007D
:1047A00000080000000800020406080A0C000102CC
:1047B00003040506000000000000000001020304DD
:1047C000060708090000000001020304081C304429
:1047D000586C800000000004040400000800000081
:1047E000080000080000000800020406080A0C0087
:1047F000010203040506081C3044586C80000000C8
:104800000004040400000800000008000008000084
:10481000000800020406080A0C0001020304050651
:104820005F6C697374006C69737420616C6C2063D5
:104830006F6D6D616E6400000004000000000000F8
:104840000800000008000000002000000000000038
:10485000081C3044586C8000000000040404000070
:10486000080000000800000800000008000204061C
:10487000080A0C0001020304050600000000000005
:104880000000002F000000000700070000147F1444
:104890007F1400242A7F2A12006264081323003642
:1048A0004955225000000503000000001C22410071
:1048B000000041221C000014083E08140008083EB5
:1048C0000808000000A060000008080808080000B0
:1048D00060600000002010080402003E5149453E7F
:1048E0000000427F4000004261514946002141459D
:1048F0004B31001814127F10002745454539003C04
:104900004A494930000171090503003649494936D1
:1049100000064949291E00003636000000005636C0
:1049200000000008142241000014141414140000A4
:104930004122140800020151090600324959513E32
:10494000007C1211127C007F49494936003E4141EA
:104950004122007F4141221C007F49494941007F9B
:1049600009090901003E4149497A007F0808087F8A
:104970000000417F4100002040413F01007F0814BA
:104980002241007F40404040007F020C027F007FB8
:104990000408107F003E4141413E007F090909069D
:1049A000003E4151215E007F0919294600464949D0
:1049B00049310001017F0101003F4040403F001F9D
:1049C0002040201F003F4038403F0063140814631C
:1049D00000070870080700615149454300007F4106
:1049E000410000552A552A55000041417F0000042E
:1049F0000201020400404040404000000102040067
:104A0000002054545478007F4844443800384444CB
:104A1000442000384444487F003854545418000857
:104A20007E0901020018A4A4A47C007F0804047875
:104A30000000447D4000004080847D00007F1028FD
:104A400044000000417F4000007C04180478007C92
:104A50000804047800384444443800FC2424241812
:104A60000018242418FC007C08040408004854544E
:104A7000542000043F444020003C4040207C001C67
:104A80002040201C003C4030403C0044281028447A
:104A9000001CA0A0A07C004464544C4414141414C2
:104AA00014140000000000000000000000000000DE
:104AB0000000000000F8000000000000003330009B
:104AC000000000100C06100C0600000000000000A2
:104AD000000040C07840C0784000043F04043F0418
:104AE0000400007088FC08300000001820FF211E20
:104AF0000000F008F000E018000000211C031E2157
:104B00001E0000F00888700000001E2123241927D1
:104B1000211010160E000000000000000000000030
:104B20000000000000E01804020000000007182048
:104B3000400000020418E0000000004020180700B8
:104B40000000404080F0804040000202010F01025E
:104B50000200000000F0000000000101011F01013F
:104B60000100000000000000000080B070000000A4
:104B70000000000000000000000000010101010130
:104B800001010000000000000000003030000000C3
:104B9000000000000000806018040060180601009A
:104BA000000000E010080810E000000F10202010A6
:104BB0000F00001010F8000000000020203F20200F
:104BC00000000070080808887000003028242221A6
:104BD000300000300888884830000018202020115C
:104BE0000E000000C02010F8000000070424243F3D
:104BF000240000F8088888080800001921202011E6
:104C00000E0000E0108888180000000F112020110D
:104C10000E0000380808C83808000000003F0000F7
:104C200000000070880808887000001C22212122E2
:104C30001C0000E010080810E000000031222211E2
:104C40000F00000000C0C000000000000030300075
:104C500000000000008000000000000080600000F4
:104C6000000000008040201008000001020408102D
:104C7000200040404040404040000404040404043C
:104C800004000008102040800000002010080402EA
:104C90000100007048080808F000000000303601EC
:104CA0000000C030C828E810E000071827242314AB
:104CB0000B000000C038E0000000203C2302022767
:104CC000382008F8888888700000203F20202011B4
:104CD0000E00C030080808083800071820202010EF
:104CE000080008F808080810E000203F20202010E5
:104CF0000F0008F88888E8081000203F20202320B3
:104D0000180008F88888E8081000203F20000300F9
:104D10000000C03008080838000007182020221EB4
:104D2000020008F808000008F808203F21010121CE
:104D30003F20000808F8080800000020203F20203D
:104D4000000000000808F8080800C08080807F008C
:104D5000000008F888C028180800203F20012638E5
:104D6000200008F8080000000000203F202020203C
:104D7000300008F8F800F8F80800203F003F003F36
:104D8000200008F830C00008F808203F200007186D
:104D90003F00E01008080810E0000F10202020104D
:104DA0000F0008F808080808F000203F2101010161
:104DB0000000E01008080810E0000F182424385004
:104DC0004F0008F8888888887000203F2000030C76
:104DD000302000708808080838000038202121227F
:104DE0001C00180808F8080818000000203F2000E0
:104DF000000008F808000008F808001F2020202004
:104E00001F000878880000C83808000007380E0125
:104E10000000F80800F80008F800033C0700073C11
:104E20000300081868808068180820302C03032CC1
:104E300030200838C800C83808000000203F200093
:104E4000000010080808C838080020382621202053
:104E50001800000000FE020202000000007F404037
:104E60004000000C30C000000000000000010638C7
:104E7000C00000020202FE000000004040407F002F
:104E80000000000004020202040000000000000014
:104E90000000000000000000000080808080808012
:104EA00080800002020400000000000000000000FA
:104EB000000000008080808000000019242222224F
:104EC0003F2008F8008080000000003F11202011E2
:104ED0000E000000008080800000000E11202020C5
:104EE0001100000000808088F800000E11202010C2
:104EF0003F200000808080800000001F22222222AC
:104F00001300008080F0888888180020203F20202F
:104F100000000000808080808000006B9494949357
:104F2000600008F8008080800000203F2100002001
:104F30003F2000809898000000000020203F2020A3
:104F40000000000000809898000000C08080807FF2
:104F5000000008F8000080808000203F24022D30EF
:104F60002000000808F8000000000020203F20205A
:104F700000008080808080808000203F20003F20D3
:104F8000003F8080008080800000203F21000020C2
:104F90003F200000808080800000001F2020202013
:104FA0001F00808000808000000080FFA120201171
:104FB0000E000000008080808000000E112020A0E4
:104FC000FF80808080008080800020203F212000A2
:104FD000010000008080808080000033242424248D
:104FE0001900008080E0808000000000001F202069
:104FF00000008080000000808000001F2020201022
:105000003F20808080000080808000010E300806F4
:10501000010080800080008080800F300C030C3005
:105020000F0000808000808080000020312E0E3133
:105030002000808080000080808080818E70180633
:10504000010000808080808080000021302C22219F
:10505000300000000000807C020200000000003FE1
:10506000404000000000FF00000000000000FF00C2
:1050700000000002027C800000000040403F000071
:10508000000000060101020204040000000000000C
:1050900000000003050911FF118905C300E000F0BD
:1050A00000F8000000000000004428FF11AA44009E
:1050B00000000000000000000000000000000000F0
:1050C00000000000000000000000000000000000E0
:1050D00000000000000000000000000000000000D0
:1050E00000000000000000000000000083013844C0
:1050F000829292740183000000000000007C44C78B
:10510000017D7D7D7D017D7D7D7D017D7D7D7D01BF
:10511000FF0000000000000100010001000100018B
:10512000000100000000000000000001010000007C
:10513000000000000000000000000000000000006F
:10514000000000000000000000000000000000005F
:10515000000000000000000000000000000000004F
:10516000000000000000000000000000010100003D
:10517000000000000101000000000000000000012C
:10518000010101010101010101010101010101010F
:1051900001000000000000000000004040404040CE
:1051A00000006D6D6D6D6D000060606060600000FE
:1051B00040404040400000000000000000000000AF
:1051C00000000000000000000000000000000000DF
:1051D00000000000000000000000000000000000CF
:1051E00000000000000000000000000000000000BF
:1051F00000000000000000000000000000000000AF
:10520000000000000000000000000000000000009E
:105210000000000000000000000000DBDBDBDBDB47
:105220000000DBDBDBDBDB0000DBDBDBDBDB0000F0
:10523000DBDBDBDBDB0000DADADADADA0000D8D835
:10524000D8D8D80000C0C0C0C0C00000C0C0C0C016
:10525000C00000C0C0C0C0C00000C0C0C0C0C0000E
:1052600000808080808000000000000000000000BE
:10527000000000000000000000000000000000002E
:10528000000000000000000000000000000000001E
:1052900000000000000000000000000606060606F0
:1052A00000000606060606000006060606060000C2
:1052B00006060606060000060606E6662000060646
:1052C0008606060000060606068600000606060696
:1052D000060000868686868680808686068686C04C
:1052E000C08686860606D0307606060606000006CC
:1052F0000606060600000606060606000006060666
:105300000606000006060606060000000000000073
:10531000000000000000000000000000000000008D
:10532000000000000000000000000000000000007D
:10533000000000000000000000000000601C00FEF3
:1053400000010200C41820029E63B20E00FF81819A
:10535000FF00008040300F00000000FF0023EAAA99
:10536000BFAAEA033F00FF000000000000000000A9
:10537000000000000000000000000000000000002D
:10538000000000000000000000000000000000001D
:10539000000000000080808000000000008080800D
:1053A00000000000000000000000000000000000FD
:1053B000000000000000000000000E0C08000001CA
:1053C0000101010100000001000000010081808056
:1053D0008180818080808001010101000000010046
:1053E000000001000101090C0E0000000000000097
:1053F00000000000000000000000C0C0C0C0C0C02D
:10540000C0C0C0C0C0C0C0C0C0C0C0C0C0C0C0C09C
:10541000C000001E21404050215E001E214040502F
:10542000215E0000000000000000000000000000FD
:10543000000000000000000000000000000000006C
:1054400000000000000000000000000000FFFFC19D
:10545000C1FFFFC1C1FFFF0000000000000000000D
:10546000000000000000000000000000000000003C
:1054700000000000000000000000FFFF80FCF3EFD0
:10548000F3FC80FF80EEEEEEF5FBFF9CBEB6B68827
:10549000FF000000B454000800000020700000006D
:1054A000101C000824550008700000202034000063
:1054B000201C00080024F400000000000000000090
:1054C00000000000000000000000000000000000DC
:1054D00000000000000000000000000000000000CC
:1054E00000000000000000000000000000000000BC
:1054F000712C00085D2D00088000002000C00120F4
:105500008020002038000020000000000000000083
:10551000000000002048000826480008C6E533B413
:045520003D1D000825
:04000005080000ED02
:00000001FF
